:100000000C940E010C9436010C9436010C943601BC
:100010000C9436010C9436010C9436010C94010DAD
:100020000C9436010C9436010C9436010C94360174
:100030000C9436010C94C10D0C9436010C943601CD
:100040000C94B70C0C9436010C94850C0C945F0C3A
:100050000C9436010C9436010C9436010C94360144
:100060000C9436010C9436014E414E494E49545978
:10007000494E46CDCCCC3D0AD7233C17B7D1387773
:10008000CC2B329595E6241FB14F0A000020410089
:1000900000C84200401C4620BCBE4CCA1B0E5AAED3
:1000A000C59D7400407A10F35A00A0724E180900E2
:1000B00010A5D4E80000E87648170000E40B5402CD
:1000C0000000CA9A3B000000E1F505000080969808
:1000D00000000040420F000000A086010000001058
:1000E0002700000000E8030000000064000000009A
:1000F000000A00000000000100000000002C76D87B
:1001000088DC674F0823DFC1DFAE59E1B1B796E560
:10011000E3E453C63AE651997696E8E6C28426EBC4
:10012000898C9B62ED407C6FFCEFBC9C9F40F2BAD7
:10013000A56FA5F490055A2AF75C936B6CF9676D6F
:10014000C11BFCE0E40D47FEF520E6B500D0ED90C4
:100150002E0300943577050080841E080000204E91
:100160000A000000C80C333333330F986E1283112A
:1001700041EF8D2114893BE65516CFFEE6DB18D101
:10018000844B381BF77C1D901DA4BBE424203284D3
:10019000725E228100C9F124ECA1E53D27005EBC1E
:1001A000E2613FDD83C29C7E20A3FD1F41009D23B1
:1001B000BE46DB65F88C11AF32CA57E97400000007
:1001C00000240027002A0000000000250028002B42
:1001D0000000000008000201000003040700000006
:1001E0000000000000000000002300260029000499
:1001F00004040404040404020202020202030303CE
:1002000003030301020408102040800102040810C7
:100210002001020408102000E80D151C11241FBE47
:10022000CFEFD8E0DEBFCDBF23E0ACE7B1E001C047
:100230001D92A23CB207E1F711E0A0E0B1E0EAE5CF
:10024000FFE402C005900D92AC37B107D9F711E079
:10025000CDE0D1E004C02197FE010E94CC22CC3039
:10026000D107C9F70E94AB0E0C94A0270C94000094
:100270008091290290912A0220912502222319F0CF
:10028000213039F008959C01220F331F820F931FF4
:100290000895880F991F0895CF93DF93C091150299
:1002A000D09116020E943801C830D10571F044F493
:1002B000C230D10591F02497A9F0DF91CF91089534
:1002C000C031D10511F0A097C1F797FD079623E043
:1002D000959587952A95E1F7F0CF97FD019695952D
:1002E0008795EBCF97FD039695958795959587957F
:1002F000E4CFFC01248135816217730720F48081EB
:100300009181009729F41092850185E891E0089584
:10031000860F971F08950895AF92BF92CF92DF92F4
:10032000EF92FF920F931F93CF93DF936C017B01AA
:100330008B01040F151FEB015E01AE18BF08C0173B
:10034000D10759F06991D601ED91FC910190F081AE
:10035000E02DC6010995892B79F7C501DF91CF9171
:100360001F910F91FF90EF90DF90CF90BF90AF90D3
:100370000895FC01538D448D252F30E0842F90E0AB
:10038000821B930B541710F0CF9608950197089590
:10039000FC01918D828D981761F0A28DAE0FBF2F59
:1003A000B11D5D968C91928D9F5F9F73928F90E0AF
:1003B00008958FEF9FEF0895FC01918D828D98171E
:1003C00031F0828DE80FF11D858D90E008958FEF5B
:1003D0009FEF0895FC01918D228D892F90E0805C24
:1003E0009F4F821B91098F73992708958CE292E0A9
:1003F0000E94EA0121E0892B09F420E0822F089570
:10040000FC01A48DA80FB92FB11DA35ABF4F2C9189
:10041000848D90E001968F739927848FA689B78980
:100420002C93A089B1898C91837080648C93938D77
:10043000848D981306C00288F389E02D80818F7D1A
:1004400080830895EF92FF920F931F93CF93DF93D2
:10045000EC0181E0888F9B8D8C8D98131AC0E88900
:10046000F989808185FF15C09FB7F894EE89FF89CF
:100470006083E889F98980818370806480839FBF6D
:1004800081E090E0DF91CF911F910F91FF90EF906D
:100490000895F62E0B8D10E00F5F1F4F0F7311277D
:1004A000E02E8C8D8E110CC00FB607FCFACFE889B8
:1004B000F989808185FFF5CFCE010E940002F1CF3E
:1004C000EB8DEC0FFD2FF11DE35AFF4FF0829FB72C
:1004D000F8940B8FEA89FB8980818062CFCFCF931C
:1004E000DF93EC01888D8823B9F0AA89BB89E8895C
:1004F000F9898C9185FD03C0808186FD0DC00FB602
:1005000007FCF7CF8C9185FFF2CF808185FFEDCF7F
:10051000CE010E940002E9CFDF91CF910895833090
:1005200081F028F4813099F08230A9F00895873065
:10053000A9F08830C9F08430B1F4809180008F7DBB
:1005400003C0809180008F7780938000089584B5E8
:100550008F7784BD089584B58F7DFBCF8091B000E7
:100560008F778093B00008958091B0008F7DF9CF90
:100570001F93CF93DF93282F30E0F901EF52FE4F06
:100580008491F901ED5FFD4FD491F901E151FE4FE6
:10059000C491CC23A9F0162F81110E948F02EC2F59
:1005A000F0E0EE0FFF1FE953FE4FA591B4918FB716
:1005B000F894EC91111108C0D095DE23DC938FBF25
:1005C000DF91CF911F910895DE2BF8CFCF93DF936A
:1005D00090E0FC01ED5FFD4F249181519E4FFC01A5
:1005E00084918823D1F090E0880F991FFC01E35497
:1005F000FE4FA591B491FC01E953FE4FC591D491F2
:1006000061110EC09FB7F8948C91E22FE0958E2374
:100610008C932881E223E8839FBFDF91CF910895D7
:100620008FB7F894EC91E22BEC938FBFF6CF3FB7E6
:10063000F8948091810190918201A0918301B09101
:10064000840126B5A89B05C02F3F19F00196A11D76
:10065000B11D3FBFBA2FA92F982F8827BC01CD010C
:10066000620F711D811D911D42E0660F771F881F6B
:10067000991F4A95D1F708958F929F92AF92BF929A
:10068000CF92DF92EF92FF926B017C010E941703E1
:100690004B015C01C114D104E104F104B9F00E94E2
:1006A0001703681979098A099B09683E7340810517
:1006B000910580F321E0C21AD108E108F10888EE23
:1006C000880E83E0981EA11CB11CE4CFFF90EF9030
:1006D000DF90CF90BF90AF909F908F900895813022
:1006E000A1F061E081E10E94B80264E670E080E080
:1006F00090E00E943C0360E081E10E94B80262E366
:1007000070E080E090E00C943C0308952FB7F894DB
:1007100060917D0170917E0180917F0190918001B7
:100720002FBF0895DC0180E0615090F09D919827E3
:10073000E92FEF70F0E0E356FE4F2491E92FE295A8
:10074000EF70F0E0E355FE4FE491822F8E27ECCF5F
:100750000895DC012C911196ED91FC91F894818122
:10076000822B81839281322F30959323928387E06D
:1007700090E00197F1F781818323818383E290E008
:100780000197F1F790817894EFECF0E03197F1F771
:10079000922381E009F480E00895FC0190810180BA
:1007A000F281E02D292F209560FF14C0F8948281FA
:1007B000822382838181892B8183A3E2B0E0119718
:1007C000F1F78281982B9283789487ED90E00197DE
:1007D000F1F70895F8948281822382838181892BA5
:1007E0008183AFEFB0E01197F1F78281982B92836C
:1007F00078948FE090E0EBCFDF92EF92FF920F932F
:100800001F93CF93DF93EC01D62EE42E08E010E087
:10081000FF24F39461E08D2D8F2109F460E0CE0177
:100820000E94CD03FF0C01501109A1F7E11010C087
:10083000F894E981FA819181888180958923818367
:10084000E981FA81928188818095892382837894D5
:10085000DF91CF911F910F91FF90EF90DF9008955E
:10086000EF92FF920F931F93CF93DF938C017B0145
:1008700040E065E50E94FC03E70188E0E80EF11C1A
:10088000699140E0C8010E94FC03CE15DF05C1F765
:10089000DF91CF911F910F91FF90EF900895FC0190
:1008A00090810180F281E02DF8948181292F20959B
:1008B0008223818378943DE743E050E0315029F171
:1008C000DA011197F1F780818923C1F3F8948281CD
:1008D000822382838181892B81837894ABE7B7E07F
:1008E0001197F1F7F894818182238183A3E1B1E02C
:1008F0001197F1F78081982381E009F080E07894E6
:10090000E3E6F6E03197F1F7089580E00895AF92BD
:10091000BF92CF92DF92EF92FF920F931F93CF93EC
:10092000DF938B01BC018091AC039091AD030E94D9
:10093000300440E06EEB8091AC039091AD030E94D7
:10094000FC03E801680189E0C80ED11CA090AC034B
:10095000B090AD0388E0E82EF12C10E001E0C50175
:100960000E94A9038111102B000F81E0E81AF10801
:10097000B1F71993CC16DD0649F78091AC0390913D
:10098000AD030E944F0491E0813009F090E0892F7F
:10099000DF91CF911F910F91FF90EF90DF90CF905B
:1009A000BF90AF9008950F931F93CF93DF938C0167
:1009B000EB018091AC039091AD030E944F04811133
:1009C00002C090E00EC0BE01C8010E9487048823C7
:1009D000C1F368E0CE010E94920391E028852813BC
:1009E000F0CF892FDF91CF911F910F910895CF9371
:1009F000DF93CDB7DEB729970FB6F894DEBF0FBEF1
:100A0000CDBFBE016F5F7F4F0E94D304882331F0BA
:100A10008D818F33A9F020F48F31A1F080E007C0E1
:100A20008F3521F08F37D1F78CE001C08BE029960C
:100A30000FB6F894DEBF0FBECDBFDF91CF91089502
:100A40008AE0F5CF89E0F3CF0F931F93CF93DF9325
:100A5000CDB7DEB729970FB6F894DEBF0FBECDBF76
:100A6000182FBE016F5F7F4F8BEF91E00E94D30480
:100A7000082F882309F46FC08091FB01803109F4AD
:100A80006AC08FE51B3039F08FE71C3021F08FE111
:100A90001A3009F48FE38D838091AC039091AD03FC
:100AA0000E944F046BEF71E08091AC039091AD0315
:100AB0000E94300440E06EE48091AC039091AD035D
:100AC0000E94FC0340E06B818091AC039091AD03E8
:100AD0000E94FC0340E06C818091AC039091AD03D7
:100AE0000E94FC038091FB01803141F040E06D8168
:100AF0008091AC039091AD030E94FC038091AC0304
:100B00009091AD030E944F046BEF71E08091AC03B4
:100B10009091AD030E9430044091A70368E4809156
:100B2000AC039091AD030E94FC0364E170E080E0AF
:100B300090E00E943C038091A703882331F06AE093
:100B400070E080E090E00E943C038091AC039091C3
:100B5000AD030E944F04802F29960FB6F894DEBF94
:100B60000FBECDBFDF91CF911F910F9108950F93CD
:100B70001F93CF93DF938C01D0E0C0E061E081E16F
:100B80000E94B80264E670E080E090E00E943C03BE
:100B900060E081E10E94B80262E370E080E090E0F2
:100BA0000E943C0321960C171D0741F7DF91CF915E
:100BB0001F910F910895CF93DF93EC0189859A855A
:100BC0002091150230911602613009F07FC0019624
:100BD0009A8789872130310509F044C0049714F0C1
:100BE0001A861986E985FA853696EE0FFF1FEC0FF7
:100BF000FD1F6081617088810E94B802E985FA85D5
:100C00003696EE0FFF1FEC0FFD1F60817181759509
:100C1000679561708A810E94B802E985FA853696E7
:100C2000EE0FFF1FEC0FFD1F6081718175956795B9
:100C30007595679561708C810E94B802E985FA8587
:100C40003696EE0FFF1FEC0FFD1F6081718193E060
:100C5000759567959A95E1F761708E81DF91CF91D7
:100C60000C94B802089714F01A861986E985FA855B
:100C70003A96EE0FFF1FEC0FFD1F608161708881B7
:100C80000E94B802E985FA853A96EE0FFF1FEC0F35
:100C9000FD1F608171817595679561708A810E94E1
:100CA000B802E985FA853A96EE0FFF1FEC0FFD1F9B
:100CB00060817181759567957595679561708C8177
:100CC0000E94B802E985FA853A96BBCF01979A87C8
:100CD00089872130310539F497FF84CF83E090E094
:100CE0009A8789877FCF97FFC1CF87E090E09A8767
:100CF0008987BCCF80910302909104022091170252
:100D000060E0211161E00C94DB0580910302909179
:100D100004022091170261E0211160E00C94DB05D0
:100D20001F93CF93DF93EC01162F0E944C01092EE5
:100D3000000CAA0BBB0BAC01BD0123E0440F551FF7
:100D4000661F771F2A95D1F7111164C0411551050F
:100D500021E062077105E0F481E080938A015093FD
:100D60008901409388018091880190918901909335
:100D700087008093860080918A0180618093810042
:100D800080E1809381001B86DF91CF911F910895B0
:100D90004115510528E06207710548F422E02093CF
:100DA0008A01BF719093890180938801DCCF41153E
:100DB000510580E46807710558F483E080938A0147
:100DC000F6E07695679557954795FA95D1F7C7CF91
:100DD00041155105610521E0720740F484E08093DC
:100DE0008A01452F562F672F7727B9CF85E080934B
:100DF0008A0141155105610584E0780740F43AE025
:100E000076956795579547953A95D1F7A8CF8FEF87
:100E10009FEFC8CF4115510521E06207710510F51C
:100E200081E080938A0150938901409388018091E9
:100E3000880190918901909387008093860080912A
:100E40008A01806180938100109281001092850058
:100E50001092840080918A0180618093810081E0FA
:100E60008B8792CF4115510528E06207710548F440
:100E700022E020938A01BF719093890180938801B9
:100E8000D6CF4115510580E46807710558F483E019
:100E900080938A0126E076956795579547952A9520
:100EA000D1F7C1CF41155105610521E0720740F42A
:100EB00084E080938A01452F562F672F7727B3CF81
:100EC00085E080938A0141155105610584E078072A
:100ED00040F48AE076956795579547958A95D1F7BE
:100EE000A2CF8FEF9FEFC8CFCF92DF92EF92FF920A
:100EF000C090C901D090CA01E090CB01F090CC0124
:100F00008091C5019091C601A091C701B091C8011F
:100F1000C816D906EA06FB0679F460E08091030260
:100F2000909104020E94900686E08093CD01FF908C
:100F3000EF90DF90CF9008958091BA01811110C099
:100F40000E947A0681E0C81AD108E108F108C0922F
:100F5000C901D092CA01E092CB01F092CC01E7CF57
:100F60000E9485068FEFC81AD80AE80AF80AEFCF60
:100F70008091AC039091AD030E944F0440E06CEC73
:100F80008091AC039091AD030E94FC034091A703B4
:100F900064E48091AC039091AD030E94FC038091C6
:100FA000A9038823A1F0E091A803E9506EEE72E056
:100FB000E33038F4F0E0EE0FFF1FE65CFE4F608197
:100FC0007181072E000C880B990B0C943C0308953B
:100FD000BF92CF92DF92EF92FF920F931F93CF9326
:100FE000DF93EC01B62EC72E8D85811105C0CE0191
:100FF0000E944F0481110EC01B861D861C8680E056
:10100000DF91CF911F910F91FF90EF90DF90CF90E4
:10101000BF90089540E060EFCE010E94FC0301E024
:10102000E12CD12C11E0CE010E94A903F82ECE01B3
:101030000E94A90391E0F91218C0813099F511348A
:10104000D8F2DB86D11002C081E08D878B818823A6
:1010500099F22396EB2DFC2DCF010896299121932F
:10106000E817F907D9F781E0CBCFEE2DF0E0F812C1
:101070000FC08B851817A0F4DE01AE0FBF1F1396AB
:101080008C91802379F4F12C193008F41C87D12E2F
:10109000EC0FFD1F8381902F9095892383830AC0D5
:1010A0008113F1CFFE01EE0DF11D8381802B83832F
:1010B000FF24F3946F2DCE010E94CD031F5F000F1C
:1010C00011F4E39401E087E08E1508F0ACCFB7CFC0
:1010D000CF93DF93EC01E091AC03F091AD03138665
:1010E000158614861286118610861782168215823E
:1010F00014821382BC018091AC039091AD030E94D5
:10110000E807982F882341F067E0CE010E94920300
:1011100091E02F81281390E0892FDF91CF910895DE
:10112000AF92BF92CF92DF92EF92FF920F931F93F5
:10113000CF93DF93CDB7DEB761970FB6F894DEBFDC
:101140000FBECDBFA0908D01B0908E01C0908F01D9
:10115000D09090018091C30175018601882351F0E0
:10116000CE010A960E946808811137C0E12CF12C4B
:101170000EEF12EC20E030E040E252ECB701C80183
:101180000E94A3221816B4F420E030E040EA52E4B2
:10119000B701C8010E94722087FF0CC0C701D801A7
:1011A00080938D0190938E01A0938F01B093900155
:1011B00057016801B501C60161960FB6F894DEBF0C
:1011C0000FBECDBFDF91CF911F910F91FF90EF9098
:1011D000DF90CF90BF90AF900895BE016F5F7F4FBB
:1011E000CE010A960E94D304882309F4BFCF6A81F6
:1011F00070E0762F6627770F770F770F298148E009
:10120000249F90011124262B372B8A858031D1F41D
:10121000688570E08F81AB01481B5109CA01969522
:10122000982F8827979587950E94B822CB014097E1
:10123000B90153E0660F771F5A95E1F760789C017A
:10124000260F371F213854EE35070CF48FCFB90124
:10125000330F880B990B0E94792020E030E040E0AA
:101260005CE30E94D8207B018C0184CFFC010190BB
:101270000020E9F73197AF01481B590BBC018CE204
:1012800092E00C948C01EF92FF920F931F93CF93F7
:10129000DF937C0105E012E0D0E0C0E0F80161914D
:1012A0008F01C7018C0F9D1F0E94A1212196C7327B
:1012B000D105A1F787E290E0DF91CF911F910F91C7
:1012C000FF90EF9008958091BB019091BC010E9426
:1012D00043091092BD010895CF93DF93C5E0D2E09A
:1012E00083E690E09983888380E797E1A0E0B0E00F
:1012F0008A839B83AC83BD8388E99AE3A0E0B0E056
:101300008E839F83A887B98780E090E0A8E4B2E449
:101310008A879B87AC87BD8784E190E09F878E8713
:1013200081E090E0998B888B1A8A1B8A8C8B95E0E0
:101330009D8B8E8B1F8A9AE0988F198E1A8E1B8E2A
:101340001C8E1D8E1E8E1F8E92E098A389A38AA3E9
:1013500023E02BA390938C0128E833E13DA32CA339
:101360008EA30E9463098A819B81AC81BD81809399
:10137000C9019093CA01A093CB01B093CC01809393
:10138000C5019093C601A093C701B093C801DF9136
:10139000CF9108950F931F93CF93DF93C5E0D2E0D1
:1013A0008C0105501240C8018C0F9D1F0E9499218D
:1013B000899382E0CC32D807B1F787E290E0DF91E1
:1013C000CF911F910F9108950F931F93CF93DF93A8
:1013D000CDB7DEB7A0970FB6F894DEBF0FBECDBF76
:1013E0001F9293E29F937F936F935F934F93282F66
:1013F000082E000C330B3F938F9382E591E09F936F
:101400008F931F9280E28F938E010F5F1F4F1F9368
:101410000F930E94F224C8010E9436090FB6F89477
:10142000DEBF0FBECDBFA0960FB6F894DEBF0FBED5
:10143000CDBFDF91CF911F910F9108950F931F930F
:10144000CF93DF93CDB7DEB7A0970FB6F894DEBF8A
:101450000FBECDBF1F9293E29F937F936F93282F70
:10146000082E000C330B3F938F938AE591E09F93F6
:101470008F931F9280E28F938E010F5F1F4F1F93F8
:101480000F930E94F224C8010E9436090FB6F89407
:10149000DEBF0FBECDBFA0960FB6F894DEBF0FBE65
:1014A000CDBFDF91CF911F910F9108950F931F939F
:1014B000CF93DF93CDB7DEB7A0970FB6F894DEBF1A
:1014C0000FBECDBF1F9293E29F937F936F93282F00
:1014D000082E000C330B3F938F9381E691E09F938E
:1014E0008F931F9280E28F938E010F5F1F4F1F9388
:1014F0000F930E94F224C8010E9436090FB6F89497
:10150000DEBF0FBECDBFA0960FB6F894DEBF0FBEF4
:10151000CDBFDF91CF911F910F910895FC01808184
:101520009181009711F00C94641C60E070E0CB0195
:101530000895CF93DF93EC0188819981009711F092
:101540000E948223198218821D821C821B821A82A9
:10155000DF91CF910895FC0180819181009711F076
:101560000C94822308950F931F93CF93DF938C01E4
:10157000EB01FC01808191810097E1F06881798124
:1015800061157105A9F0428153812C813D8142177B
:10159000530770F00E94DC248C819D81F8019583B3
:1015A00084831D821C82DF91CF911F910F9108953A
:1015B0000E94822388819981F801918380838A81A6
:1015C0009B81938382838C819D81958384831982FF
:1015D00018821B821A82E5CF0F931F93CF93DF935C
:1015E000EC0188819981009759F02A813B81261767
:1015F000370730F081E0DF91CF911F910F9108956F
:101600008B016F5F7F4F0E940B24009759F09983E5
:1016100088831B830A832C813D81232B59F7FC018E
:101620001082E8CF80E0E7CFEF92FF920F931F93F5
:10163000CF93DF93EC017B018A01BA010E94EC0A8F
:1016400081110BC0CE010E94990ACE01DF91CF918A
:101650001F910F91FF90EF9008951D830C83B701A8
:10166000888199810E94DC24F0CFFC0111821082D4
:10167000138212821582148250E040E06AE671E023
:101680000C94140BFB0101900020E9F73197AF0196
:10169000461B570B0C94140BAF92BF92CF92DF9264
:1016A000EF92FF920F931F93CF93DF936C015B0137
:1016B0007A0189012417350720F48F2D7901042F31
:1016C000182FC6010E94350BD5011496CD91DC91DF
:1016D000EC16FD06E0F40C171D0708F4E801D5012F
:1016E000ED91FC911197EC0FFD1F108110826D910F
:1016F0007C916E0D7F1DC60161157105A1F00E94E0
:10170000420BF50180819181C80FD91F1883C60152
:10171000DF91CF911F910F91FF90EF90DF90CF90CD
:10172000BF90AF9008950E94990AEBCFCF93DF93BB
:10173000EC01FB018617970749F060817181611503
:10174000710541F0448155810E94140BCE01DF9157
:10175000CF9108950E94990AF9CFFF920F931F939A
:10176000CF93DF93CDB7DEB728970FB6F894DEBFDF
:101770000FBECDBF86E0F82E8CE292E00E94EA0117
:10178000892B09F48AC08CE292E00E94C801182FCC
:10179000833251F08A3309F049C06AE671E087E983
:1017A00093E00E94420BE8CF2091A1033091A20365
:1017B0008091A5039091A60328173907ECF6409174
:1017C000A3035091A40320919F033091A003C9016A
:1017D00001969093A00380939F03F29EC001F39E15
:1017E000900D112467E973E0840F951F0E94960BFA
:1017F0008091A1039091A20301969093A2038093FC
:10180000A10380919F039091A0032091A5033091A3
:10181000A603281739070CF0AFCF2F5F3F4F821B6D
:10182000930B9093A00380939F03A6CF1A821982F3
:101830001C821B821E821D8267E973E0CE01019625
:101840000E94960B1F8318860D811E810F5F1F4F0C
:10185000B801CE0101960E94EC0A8823C9F02981C3
:101860003A818D819E81BE01695F7F4F820F931FF8
:101870000E94DC241E830D83BE016F5F7F4F87E9CA
:1018800093E00E94960BCE0101960E94AB0A74CFA2
:10189000CE0101960E94990AEFCF28960FB6F894D0
:1018A000DEBF0FBECDBFDF91CF911F910F91FF9093
:1018B00008950E94F60181110C94AD0B08951F92BA
:1018C0000F920FB60F9211242F933F934F935F9374
:1018D0006F937F938F939F93AF93BF93EF93FF93F8
:1018E0008CE292E00E940002FF91EF91BF91AF91D4
:1018F0009F918F917F916F915F914F913F912F9128
:101900000F900FBE0F901F9018951F920F920FB659
:101910000F9211242F938F939F93EF93FF93E09156
:101920003C02F0913D028081E0914202F09143023D
:1019300082FD1BC09081809145028F5F8F73209143
:101940004602821741F0E0914502F0E0E45DFD4F70
:10195000958F80934502FF91EF919F918F912F91E9
:101960000F900FBE0F901F9018958081F4CF1F929B
:101970000F920FB60F9211242F933F938F939F9343
:10198000AF93BF9380917D0190917E01A0917F01E3
:10199000B091800130917C0123E0230F2D3758F561
:1019A0000196A11DB11D20937C0180937D01909330
:1019B0007E01A0937F01B09380018091810190917D
:1019C0008201A0918301B09184010196A11DB11DF6
:1019D0008093810190938201A0938301B09384014D
:1019E000BF91AF919F918F913F912F910F900FBE1B
:1019F0000F901F90189526E8230F0296A11DB11D88
:101A0000D2CF1F920F920FB60F9211242F933F93B4
:101A10004F935F936F937F938F939F93AF93BF93F6
:101A2000CF93DF93EF93FF932091C90230E0F90148
:101A3000EF52FE4F8491F901ED5FFD4FD491F90112
:101A4000E151FE4FC491CC2379F081110E948F02A5
:101A5000EC2FF0E0EE0FFF1FEB51FE4FA591B4917C
:101A6000EC91ED2381E009F480E02091CC023091EB
:101A7000CD022F5F3F4F3093CD022093CC02909147
:101A80009603943618F095E09093CA029091CA029A
:101A9000933009F44CC0E0F4923011F19091CB02F4
:101AA000992319F081116BC02D9AFF91EF91DF916D
:101AB000CF91BF91AF919F918F917F916F915F91E6
:101AC0004F913F912F910F900FBE0F901F9018953F
:101AD000943009F448C0953009F78111DFCF09C06F
:101AE0008111DCCF2091CC023091CD02243631051A
:101AF00028F41092CD021092CC02D0CF109296030F
:101B0000E091960391E09E0F90939603F0E0209170
:101B1000CC023091CD02EE0FFF1FE753FD4F36830D
:101B200025831092CD021092CC0293E019C081302F
:101B300009F0B4CFE091960391E09E0F9093960345
:101B4000F0E02091CC023091CD02EE0FFF1FE75361
:101B5000FD4F368325831092CD021092CC0294E083
:101B60009093CA029BCF882359F22091CC023091E6
:101B7000CD022536310508F491CF95E0F1CF2D98AF
:101B800094CF1F920F920FB60F9211242F933F9371
:101B90004F935F936F937F938F939F93AF93BF9375
:101BA000EF93FF93E0918601F09187010995FF91F2
:101BB000EF91BF91AF919F918F917F916F915F91C5
:101BC0004F913F912F910F900FBE0F901F9018953E
:101BD000EF92FF920F931F93CF93DF9310922F02F8
:101BE00010922E0288EE93E0A0E0B0E080933002E5
:101BF00090933102A0933202B093330284E491E0D7
:101C000090932D0280932C0285EC90E09093390202
:101C10008093380284EC90E090933B0280933A02E8
:101C200080EC90E090933D0280933C0281EC90E048
:101C300090933F0280933E0282EC90E090934102A9
:101C40008093400286EC90E090934302809342029E
:101C500010924502109246021092470210924802DA
:101C600060E082E00E94E602E5E0F2E0E491E093C9
:101C7000AE03E1EFF1E0E491F0E0EE0FFF1FEB5176
:101C8000FE4F859194919093B0038093AF0310928F
:101C9000B9031092BB031092BA031092B8031092CA
:101CA000B7031092B6031092B5031092B4031092CA
:101CB000B3031092B2031092B1038EEA93E09093B3
:101CC000AD038093AC031092AB031092A70389E09D
:101CD0008093A80381E08093A9038093AA031092C4
:101CE0009E0310929D031092A00310929F031092E6
:101CF000A2031092A10384E090E09093A603809346
:101D0000A50380E290E00E94E622EC0125E030E0AD
:101D1000299339937E018C01005E1F4FC7010E94F9
:101D2000350B86E0E80EF11CE016F106B9F7D0930A
:101D3000A403C093A30387E993E00E94350B89E0D5
:101D40008093C9021092CB02DF91CF911F910F9126
:101D5000FF90EF900895CF93DF93CDB7DEB7C754D0
:101D6000D1090FB6F894DEBF0FBECDBF789484B50D
:101D7000826084BD84B5816084BD85B5826085BD87
:101D800085B5816085BD80916E00816080936E0015
:101D90001092810080918100826080938100809107
:101DA00081008160809381008091800081608093B8
:101DB00080008091B10084608093B1008091B00078
:101DC00081608093B00080917A00846080937A0073
:101DD00080917A00826080937A0080917A0081609D
:101DE00080937A0080917A00806880937A001092C4
:101DF000C100E0913C02F0913D0282E08083E091DD
:101E00003802F09139021082E0913A02F0913B02DF
:101E10008FEC808310924402E0914002F0914102E5
:101E200086E08083E0913E02F0913F0280818061F4
:101E30008083E0913E02F0913F0280818860808340
:101E4000E0913E02F0913F02808180688083E091C2
:101E50003E02F0913F0280818F7D80838CE292E090
:101E60000E94EA01892B29F08CE292E00E94C801CD
:101E7000F5CF61E081E10E94E60281E08093CE012E
:101E80001092C3011092B6011092BE011092BD01D2
:101E90001092C4011092BC011092BB0110E000E04E
:101EA000C8010E94CA0980910502909106028336FA
:101EB000910529F51093BC010093BB01C8010E9454
:101EC000CA091092060210920502C8010E94430935
:101ED0008091BB019091BC018796863F23E09207D9
:101EE0000CF0ABC09093BC018093BB0183E690E003
:101EF00090930602809305020E94630908C0095D61
:101F00001F4F063F33E0130759F60E946C0980E02B
:101F100090E0A0E9B1E480938D0190938E01A093AD
:101F20008F01B09390011092C3011092B5010E94ED
:101F300086036093BF017093C0018093C1019093A9
:101F4000C20160E082E00E94E602E091AC03F09101
:101F5000AD031386158614861286118610861782A5
:101F600016821582148213821092AB0301E0BE0127
:101F70006F5D7F4F8091AC039091AD030E94E807A5
:101F8000882309F469C067E0CE0181960E9492031C
:101F900098A58913ECCF8091A703811128C0809167
:101FA000AC039091AD030E944F04BE016F5D7F4F63
:101FB0008091AC039091AD030E94300440E064EB4B
:101FC0008091AC039091AD030E94FC038091AC031F
:101FD0009091AD030E94A903182F8091AC039091BA
:101FE000AD030E944F04111102C00093A70380911A
:101FF000AC039091AD030E944F04882339F0BE01D9
:102000006F5F7F4FCE0181960E9487041091A803D5
:1020100089A1803111F40C948B1BCE0181960E9412
:10202000F704811778F48091A8038093A803809126
:10203000AB038F5F8093AB039ACF1092BC011092D9
:10204000BB0154CF89A1803111F48CE0EECFCE01D9
:1020500081960E94F704E9CF8BEF91E00E94680817
:10206000882341F081E08093C3018AE00E94240527
:102070000E94B8078091C301813011F40E9490083A
:1020800080912802811106C083E08093280282E0BB
:1020900080938C01809121028093BA0184E390E0C7
:1020A0000E94E6228C0189E8D80118968C93189733
:1020B00088E0E2E2F1E01C9601900D928A95E1F74A
:1020C00080E1EAE2F1E0D801549601900D928A9500
:1020D000E1F780E1EAE2F1E0D801949601900D92F7
:1020E0008A95E1F784E090E0F8019183808385E0B0
:1020F00090E09383828386E090E09583848387E0F9
:1021000090E09783868358014801F8E08F0E911C78
:102110006801D6018C91B2E0CB0ED11C61E00E9427
:10212000E6028C149D04A9F7F801128611868091AD
:1021300015029091160202970CF079C181E090E0AF
:102140009093160280931502D8011B961C9210934F
:102150000402009303028091180281110BC0F50163
:102160008081F2E0AF0EB11C60E00E94B802AC14B6
:10217000BD04A9F78091070290910802A09109027D
:10218000B0910A028093C5019093C601A093C70144
:10219000B093C8018093C9019093CA01A093CB0169
:1021A000B093CC01FF24F394F092BD0180E18093C1
:1021B00081001092800084E080938A0182E19AE796
:1021C0009093890180938801909387008093860083
:1021D00084E18093810084E797E090938701809366
:1021E0008601F0926F0060E0C8010E949006F894AA
:1021F00082E08093B0008093B10094E69093B300A6
:102200001092B2008093700078948093CA0210926A
:1022100096038091C90260E00E94E602F092B70145
:1022200061E081E10E94B80268EC70E080E090E03B
:102230000E943C0360E081E10E94B8021092CD014F
:10224000FF24F3949E012F5F3F4F69018091F301BA
:1022500081110CC00E9486036093EF017093F0011E
:102260008093F1019093F201F092F3018091E701E4
:1022700081110CC00E9486036093E3017093E40116
:102280008093E5019093E601F092E7018091DB01F4
:10229000811104C00E948603F092DB018091D3017A
:1022A00081110CC00E9486036093CF017093D0010E
:1022B0008093D1019093D201F092D301F092CE019C
:1022C0008091A1039091A203181619060CF01CC16D
:1022D000CE01C6960E94350BCE01C0960E94350BEA
:1022E0008091A1039091A203009709F405C10CF01D
:1022F000A1C0CE0181960E94350BBE016F5D7F4F5C
:10230000CE01C6960E94B30ACE0181960E94AB0A06
:1023100022E030E050E040E0BE016A5C7F4FC60141
:102320000E944C0BC6010E948E0A4B01C6010E94FE
:10233000AB0A2AAD3BAD42E050E0BE016A5C7F4F84
:10234000C6010E944C0BB601CE01C0960E94B30A92
:10235000C6010E94AB0AF401E336F10508F0CCC0D7
:10236000EC54FE4E0C94CC22641270127712A01220
:10237000A412C712F51205133E137C124813521310
:1023800057138013851395139D13A013A313AF1335
:10239000DB13EB13F0130314141419141E14241478
:1023A00037144B14511461149A149F14AF14BA14B7
:1023B000C714D314D814DD1401157C12E7140415C6
:1023C0007C127C127C127C120915221526157C12B7
:1023D0007C122A157C122F1535157C127C127C126A
:1023E0007C125415601565156A159915AC15B11553
:1023F000C215C715CC15D315DA15DF15EB15F01579
:10240000FC15011608160D16141619167C121D1649
:102410007C127C127C122216271633167C127C1238
:10242000391673167C12D3167C127C12D71682E0F2
:1024300090E086CE20919D0330919E0346E0429F1E
:10244000C001439F900D11246091A3037091A403D8
:10245000680F791F1A8219821C821B821E821D82BC
:10246000C6010E94960B80919D0390919E03019658
:1024700090939E0380939D032091A1033091A2032A
:10248000215031093093A2032093A1032091A50389
:102490003091A6032817390744F42F5F3F4F821B62
:1024A000930B90939E0380939D031AA219A21CA2E2
:1024B0001BA21EA21DA2B601CE0181960E94B30AE4
:1024C000C6010E94AB0A19CF4091C9015091CA01BF
:1024D0006091CB017091CC0180E50E94E4090CC0B1
:1024E0006091C40170E089E40E941E0A05C068E69C
:1024F00071E085E40E94560ACE01C0960E94AB0AA4
:10250000CE01C6960E94AB0A8091C9019091CA0182
:10251000A091CB01B091CC01E091CD01E93010F058
:102520000C94851BF0E0E956FD4E0C94CC22E3168A
:10253000B81AEC1A091B1F1B1D1B2B1B371B611B19
:1025400068E171E086E4D6CF88E191E09F938F93B4
:102550001F928AE08F931F928DE08F9380E091E02D
:102560009F938F938BE691E09F938F931F9280E2CE
:102570008F93DF92CF920E94F224B60186E40E94EC
:10258000560A0FB6F894DEBF0FBECDBFB5CF80910F
:10259000C4018111B1CF8091CE01813009F0ACCF5F
:1025A000CE01C0960E948E0A97FF03C060E070E0E3
:1025B000CB0100910B0210910C0220910D02309181
:1025C0000E02601771078207930714F48B019C01B8
:1025D0000093C5011093C6012093C7013093C80131
:1025E000F092BD01F092C40187CF60918D0170918E
:1025F0008E0180918F0190919001860122E042E04E
:102600000E94421CB6018AE575CFCE01C0960E9499
:102610008E0AAB01BC0141389AE1590796E069077F
:10262000710524F040E85AE166E070E08091C9014C
:102630009091CA01A091CB01B091CC018115E4E049
:102640009E07A105B10524F480E094E0A0E0B0E08D
:1026500084179507A607B70714F4DB01CA01809316
:102660000B0290930C02A0930D02B0930E02F09215
:10267000BD0182E090E00E94B7053ECF40910B0281
:1026800050910C0260910D0270910E028DE425CFE5
:1026900040910B0250910C0260910D0270910E025C
:1026A00089E51BCF6091180270E08FE41DCF70E0C8
:1026B00060E0CE01C0960E947901DC018C918053CC
:1026C00080931802813049F461E070E080E090E08E
:1026D0000E943C03F092BD010FCF009103021091C4
:1026E00004025801B8E0AB0EB11CF80180810E5F06
:1026F0001F4F60E00E94B802A016B106B1F7EACF02
:102700006091170270E082E5EFCE8091C4018111E3
:10271000F3CE70E060E0CE01C0960E947901DC014A
:102720008C91805380931702D5CFCE01C0960E9422
:102730008E0A637060932502CDCFF0921902CACF42
:1027400010921902C7CF70E060E0CE01C0960E94DF
:102750007901FC018081805380931B02BBCF88A943
:1027600099A9009761F4812C912C540180920F0259
:1027700090921002A0921102B0921202ABCF0E946E
:10278000601C4B015C0120E030E0A9010E94722036
:1027900087FDE9CF20E030E048EC52E4C501B40108
:1027A0000E94A322181614F7812C912CE8ECAE2E6F
:1027B000E2E4BE2EDBCFCE01C0960E948E0A6930C5
:1027C00008F469E0862F6D3008F08CE080931D02DC
:1027D0000E9424057FCF60911D0270E081E584CEC8
:1027E000CE01C0960E948E0A693EF3E07F0714F086
:1027F00068EE73E077FF02C070E060E0709314024F
:102800006093130267CF8091C301882309F474CECB
:1028100070E060E0CE01C0960E947901DC018C91ED
:1028200080538093B50156CF6091B50170E081E38C
:102830005BCE6091C30170E081E456CE60911302DB
:102840007091140282E450CE8091C9019091CA0126
:10285000A091CB01B091CC018093C5019093C601AA
:10286000A093C701B093C8011092C40133CF8091E7
:10287000C401811141CE8091CE01813009F03CCE5E
:102880001092C5011092C6011092C7011092C801A2
:102890008093C40131CE609115027091160283E5D8
:1028A00023CECE01C0960E948E0A81E090E0623075
:1028B000710514F082E090E0909316028093150267
:1028C00009CF8091C401811105CFCE01C0960E942D
:1028D0008E0A97FF03C060E070E0CB0100910B020D
:1028E00010910C0220910D0230910E0260177107B9
:1028F0008207930714F48B019C0100930702109345
:1029000008022093090230930A020093C501109334
:10291000C6012093C7013093C8010093C9011093E9
:10292000CA012093CB013093CC0182E090E00E9459
:10293000B705D0CE60911B0270E085E5D5CD6091E2
:102940000F02709110028091110290911202860183
:1029500022E042E00E94421CB60184E5CBCD2091EA
:102960001A0288EE93E0289FB001299F700D112470
:1029700088E5BACDCE01C0960E948E0A623008F476
:1029800062E0683008F067E060931A02A3CE70E05E
:1029900060E0CE01C0960E947901FC0180818053E5
:1029A0008093260297CE6091260270E084E49CCD4D
:1029B0006091190270E082E697CD4091C501509177
:1029C000C6016091C7017091C8018EE486CD0E9456
:1029D0006C098091070290910802A0910902B091C0
:1029E0000A028093C5019093C601A093C701B093DA
:1029F000C8018093C9019093CA01A093CB01B09301
:102A0000CC010C94000078CD6091250270E083E445
:102A10006BCD83E690E0909306028093050280914F
:102A2000C9019091CA01A091CB01B091CC018093D2
:102A3000070290930802A0930902B0930A020E9431
:102A400063095ACD64E771E081E654CD70E060E03F
:102A50008CE64ACD60918C0170E084E245CD6091B6
:102A6000290270912A0280E33FCDCE01C0960E94D8
:102A70008E0A6032F3E07F078105910520F460E261
:102A800073E080E090E0DC01CB01813E2EE2920712
:102A9000A105B10520F080EE9EE2A0E0B0E09093A9
:102AA0002A028093290216CE70E060E0CE01C09623
:102AB0000E947901DC018C91805380931C020ACE24
:102AC00060911C0270E08CE40FCD60918B0170E08E
:102AD00088E40ACD8091C40181110ECD8091CE0190
:102AE000813009F009CD8090C9019090CA01A09071
:102AF000CB01B090CC01CE01C0960E948E0A860E0A
:102B0000971EA81EB91EB7FE03C0812C912C54013C
:102B100000910B0210910C0220910D0230910E02D7
:102B200080169106A206B3060CF052CD95018401E1
:102B30004FCD1091CE01113009F0DECC70E060E095
:102B4000CE01C0960E947901FC0180818053809360
:102B5000BE011093BD01D0CC6091BE0170E08BE44A
:102B6000C3CC1091CE01113009F0C6CC70E060E00A
:102B7000CE01C0960E947901DC018C918053809334
:102B8000B601E7CF6091B60170E086E5ADCC60910B
:102B9000270270E08FE3A8CCCE01C0960E948E0A77
:102BA0006093270297CDCE01C0960E948E0A609353
:102BB0001E0290CD60911E0270E083E395CC70E020
:102BC00060E0CE01C0960E947901FC0180818053B3
:102BD000809322027FCD6091220270E084E384CC56
:102BE00070E060E0CE01C0960E947901DC018C911A
:102BF0008053809323026ECD6091230270E085E3C1
:102C000073CCCE01C0960E948E0A60931F0262CDE3
:102C100060911F0270E086E367CCCE01C0960E94EF
:102C20008E0A6093200256CD6091200270E087E307
:102C30005BCC70E060E088E357CC6091C30170E04A
:102C400083E652CC6091240270E08BE64DCC70E0BC
:102C500060E0CE01C0960E947901FC018081805322
:102C60008093240237CDF092CE0161E070E089E3D9
:102C70003BCC20918C01211103C0109228023CCC46
:102C800030E08CA99DA92817390784F450E040E072
:102C9000BE01605D7F4FC6010E944C0BB601CE01A4
:102CA000C0960E94B30AC6010E94AB0AB12CA12CA7
:102CB00010E000E08CA99DA9A816B9068CF4000FBD
:102CC000111FB501CE01C0960E947901DC018C91E3
:102CD000813311F40F5F1F4FBFEFAB1ABB0AEACF6E
:102CE00000932802F7CC8AE0F60111928A95E9F761
:102CF00080918C01811105C080E38983B6018CE647
:102D0000F9CB809128021BA61AA61DA61CA61FA6F9
:102D10001EA642E0BE016F5D7F4F90E00E94A01CA6
:102D2000BE016F5D7F4FCE018A960E94420B0EA5B9
:102D30001FA50115110561F0AAA4BBA461E370E011
:102D4000C5010E94D124AC014A195B09892B11F4F9
:102D50004FEF5FEF9801BE01665D7F4FCE01819618
:102D60000E944C0B0DA11EA10F3F100721F0011571
:102D7000110571F41982B6018CE60E94560ACE0143
:102D800081960E94AB0ACE018A960E94AB0AB4CB10
:102D900069A17AA1A801C6010E94E324F601E00F0F
:102DA000F11F1082E8CF70E060E08EE69DCBCE018F
:102DB000C0960E948E0A613019F460932B028ACC6F
:102DC00010922B0287CC4091C5015091C6016091B1
:102DD000C7017091C80184179507A607B707F1F1DD
:102DE000F092C401009103021091040261E070E0CE
:102DF00080E090E00E943C0360E0C8010E949006E1
:102E0000F092CD018091C9019091CA01A091CB01AE
:102E1000B091CC0140910B0250910C0260910D02D7
:102E200070910E02481759076A077B0729F0892B12
:102E30008A2B8B2B09F06CC48091B701813031F45F
:102E400082E090E00E94B7051092B7010E94F6015F
:102E5000882309F4FBC90E94AD0BF2C91092C4018A
:102E60008091C301813009F0FBC00E9486032B01D1
:102E70003C014092CF015092D0016092D1017092FA
:102E8000D2018091BF019091C001A091C101B09188
:102E9000C201B301A201481B590B6A0B7B0B493ECF
:102EA00053406105710530F4481659066A067B06E1
:102EB00008F0D6C01091B50180919B01811104C02A
:102EC00010939A01F0929B0180919A01811771F001
:102ED00010939A01113051F40E949008609396016A
:102EE00070939701809398019093990100919501B7
:102EF000002309F46EC00E949008609391017093C2
:102F0000920180939301909394010F250093950172
:102F1000113009F09DC08091960190919701A09188
:102F20009801B091990128968CAF9DAFAEAFBFAF1D
:102F300028978091910190919201A0919301B09175
:102F400094018CAF9DAFAEAFBFAF9C01AD01289691
:102F50006CAD7DAD8EAD9FAD28970E9400220E9482
:102F60006D22672B09F474C08091C5019091C60150
:102F7000A091C701B091C80124968CAF9DAFAEAFB0
:102F8000BFAF24978090130290901402092C000C7C
:102F9000AA08BB08809124022CAD3DAD4EAD5FADBB
:102FA00081111AC028966CAD7DAD8EAD9FAD28976E
:102FB0000E94A3221816D4F424968CAD9DADAEAD1C
:102FC000BFAD249788199909AA09BB094C015D0175
:102FD00017C00E94B80799CF28966CAD7DAD8EAD15
:102FE0009FAD28970E94A322181634F724968CAD23
:102FF0009DADAEADBFAD2497880E991EAA1EBB1E17
:1030000080910B0290910C02A0910D02B0910E02E2
:1030100088169906AA06BB0614F4D501C401B7FFA9
:1030200003C080E090E0DC018093C5019093C6016D
:10303000A093C701B093C8018CAD9DADAEADBFAD3F
:103040008093960190939701A0939801B093990172
:103050004092BF015092C0016092C1017092C201C2
:103060008091CE01813009F091C18091B50181112B
:103070006BC18EEC92E09093B2018093B10100910C
:10308000960310E01093B4010093B3018091CA023B
:10309000853009F059C18091D0029091D1028858B1
:1030A00091098D35910508F0A2C080919603843076
:1030B00009F06FC08091D2029091D3028097479718
:1030C00008F067C08091D4029091D50209970997C2
:1030D00008F05FC01092B0011092AF018FEF9FEF28
:1030E000DC018093AB019093AC01A093AD01B09350
:1030F000AE0181E090E09093A8018093A7018091B8
:10310000AB019091AC01A091AD01B091AE018F3FA8
:10311000EFEF9E07AE07BE0709F081C18091A301C2
:103120009091A401A091A501B091A6018093AB015B
:103130009093AC01A093AD01B093AE018091A30137
:103140009091A401A091A501B091A6012091C40184
:10315000213009F0EEC28533F1EE9F07F7E9AF07A2
:10316000F1E0BF0709F0E5C28091C9019091CA0161
:10317000A091CB01B091CC018093C5019093C60181
:10318000A093C701B093C8011092C4012093BD0160
:10319000DBC080919603843450F18091D2029091EB
:1031A000D302825491098E9710F530E020E080E040
:1031B00090E0DC01F901EC52FD4F40815181495012
:1031C00051094930510598F4F901EA52FD4F408107
:1031D0005181465151094131510508F484C0408163
:1031E0005181465051094730510508F48EC00630D0
:1031F00011050CF4A4C039EC632E32E0732EA3E069
:10320000B0E02296BFAFAEAF229745EC842E4DE9D9
:10321000942E4CE1A42E41E8B42E2296EEADFFADE3
:103220002297E017F1070CF075C0D3011B966D9142
:103230007C911C971796ED91FC91FDAFECAF90E05F
:1032400080E00E9477201B012C012CAD3DADB9011F
:1032500090E080E00E9477206CAF7DAF8EAF9FAF93
:103260002DEC3CEC4CE45FE30E94D8209B01AC01C8
:10327000C201B1010E947220F0E0E0E087FD16C0BB
:103280002DEC3CEC4CE45FE3C201B1010E94D8207C
:103290009B01AC016CAD7DAD8EAD9FAD0E947220E7
:1032A000E2E0F0E087FD02C0E1E0F0E0A50194017A
:1032B00063E971E080E091E00E94A8224F01FF0FD6
:1032C000AA08BB0886269726A826B92622968EAD80
:1032D0009FAD2297019622969FAF8EAF229792E0E4
:1032E000690E711C9ACF880F991FAA1FBB1F81609E
:1032F0002C5F3F4F2038310509F05CCF20E230E0F1
:103300003093B0012093AF01ECCE880F991FAA1F14
:10331000BB1FEECF8092AB019092AC01A092AD01A9
:10332000B092AE0180E290E09093B0018093AF0143
:10333000AFEFBFEFB093A801A093A701E0CE82E06A
:103340008093CA02109296038091BE018130F1F4FD
:103350008091C5019091C601A091C701B091C801AB
:103360002091B6012111E9C00197A109B109B7FF68
:1033700003C080E090E0DC018093C5019093C6011A
:10338000A093C701B093C801F092BD018091BD0127
:10339000813009F037CD0E9486030091E30110913E
:1033A000E4012091E5013091E6014B015C01801AB6
:1033B000910AA20AB30A41E1841647E29406A104E5
:1033C000B10430F4601771078207930708F01ACD33
:1033D0006093E3017093E4018093E5019093E6012B
:1033E00083E690E090930602809305028091C901E4
:1033F0009091CA01A091CB01B091CC0180930702BA
:1034000090930802A0930902B0930A028091BB0135
:103410009091BC010E9443091092BD01F3CC8093AE
:10342000A3019093A401A093A501B093A60186CE19
:103430001092250281E090E00E94B70502C0F09250
:10344000250290E080E022E02093CA0210929603C9
:1034500097FF50C0092E000CAA0BBB0B4091C9016D
:103460005091CA016091CB017091CC01840F951FDE
:10347000A61FB71FB7FF03C080E090E0DC01809378
:10348000C5019093C601A093C701B093C801F09203
:10349000BD015ACF80912B020E946F038FEF9FEFE7
:1034A000D2CF80912B020E946F0386EF9FEFCBCF8C
:1034B00080912B020E946F038AE090E0C4CF80913C
:1034C0002B020E946F0384E690E0BDCF1092C501ED
:1034D0001092C6011092C7011092C8011092C90142
:1034E0001092CA011092CB011092CC01AACF82E3B4
:1034F00090E0A9CF009759F2092E000CAA0BBB0B44
:103500000091C9011091CA012091CB013091CC01E9
:1035100040910B0250910C0260910D0270910E02CD
:10352000800F911FA21FB31F481759076A077B0717
:103530000CF0A5CFDB01CA01A2CF0196A11DB11DE0
:1035400040910B0250910C0260910D0270910E029D
:1035500084179507A607B70714F4AC01BD01409383
:10356000C5015093C6016093C7017093C8010CCF89
:10357000F092C4014091C5015091C6016091C7010C
:103580007091C801481759076A077B07D4F4109255
:10359000BA0180911F028093B90180912202809329
:1035A000B8018091BA0190912102981799F09091F9
:1035B000B801913079F48093210282E08093CD01AB
:1035C00021CCF092BA01809120028093B9018091C0
:1035D0002302E5CF83E0F2CF1091B9011123D1F39B
:1035E0008091BA01811112C00E947A060E943801AE
:1035F0008230910538F0880F991F880F991F059721
:103600000197F1F711501093B901FCCB0E94850688
:10361000EDCF0091030210910402D8011B968C910A
:103620008111F0CB61E070E080E090E00E943C030B
:1036300061E0C8010E949006E5CB84E0BFCF0E9404
:1036400086036093EF017093F0018093F1019093F2
:10365000F20186E0B3CF0E9486036093EF0170937E
:10366000F0018093F1019093F20187E0A7CF0E94CF
:1036700086038090EF019090F001A090F101B0904E
:10368000F2012B013C01481859086A087B08009197
:103690001E0210E030E020E0041515052605370570
:1036A00030F0681579058A059B0508F0ABCB60936F
:1036B000EF017093F0018093F1019093F20188E0A3
:1036C0007DCF80911802811112C0009103021091E8
:1036D00004025801B8E0AB0EB11CF80180810E5F06
:1036E0001F4F60E00E94B802A016B106B1F7109219
:1036F000C401F092BD010E9486036093E3017093C0
:10370000E4018093E5019093E6011092CD017ACB1C
:10371000F092B7019BCB1D3010F00C9413100C9459
:10372000251082E08093CA02109296038EEC9FEFE0
:1037300091CE8F3BF0E49F07FEEFAF07F1E0BF07AC
:1037400009F4AFCE9CF58D3139EF930737E9A30724
:1037500031E0B30709F473CEA4F48D33E9ED9E078D
:10376000E7E9AE07E1E0BE07E1F28D32994EA749E5
:10377000B14009F4BCCE82E08093CA021092960355
:1037800086CE87312FEF920727E9A20721E0B20703
:1037900009F49CCE8F3D9042AE4FB14061F78091CD
:1037A0002B020E946F038CE99FEF4DCE873848E7CC
:1037B00094074EEFA40741E0B40709F46BCEB4F4CC
:1037C000873BF8E49F07FEEFAF07F1E0BF0709F47E
:1037D0002FCE873A9845AE4FB14069F682E080938C
:1037E0002502F092270282E090E026CE8F3530EA63
:1037F00093073EEFA30731E0B30709F460CE8F33A0
:1038000040EC94074EEFA40741E0B40709F450CE12
:103810008F379048AE4FB14009F0ADCF80912B0269
:103820000E946F0381E090E00ECECF93DF9387E993
:1038300093E00E94AB0AC091A303D091A403209708
:10384000F1F0FE0132972081318146E0429FC001B4
:10385000439F900D1124C80FD91F9E018091A3038F
:103860009091A40326978217930721F0CE010E941E
:10387000AB0AF3CF0297DF91CF910C948223DF91B3
:10388000CF910895EF920F931F93CF93DF93E801A9
:1038900034E047FD34E1042E000C550B57FF03C004
:1038A000519541955109E32E022F242FAE010E941C
:1038B000BA1CCE01DF91CF911F910F91EF90089527
:1038C000662777270C94191E1F93FC0199278827D8
:1038D000BC01E89411911032E9F3193010F01E3058
:1038E000C8F31B3251F01D3249F4689406C00E949F
:1038F0008B1C610F711D811D911D119110531A3088
:10390000B0F33EF490958095709561957F4F8F4F01
:103910009F4F1F910895592F482F372F262F660F3D
:10392000771F881F991F660F771F881F991F620FC7
:10393000731F841F951F660F771F881F991F089597
:10394000BB27FB015527AA27880F991FAA1FA41779
:1039500010F0A41B83955051B9F7A05DAA3308F06D
:10396000A95DA193009779F7B111B1931192CB01A1
:103970000C946220A9E0B0E0E0ECFCE10C94C021E2
:103980006A01F22EB02E102FFBE3AF2EA01608F422
:103990001BE31F5F012F27E0AE014F5F5F4F0E94C7
:1039A000691FBC018981982F9970913009F43FC03B
:1039B0009BE2E1FC04C09E2D9170E0FC3AC05E2DBC
:1039C0005071E82FE87083FF46C084E0911101C078
:1039D00083E0EF2DE81B8F1508F0E0E0D6018E2F75
:1039E00020E2552351F1992329F0D6019C93C60179
:1039F00001966C0196012D5F3F4FE2FE24C08EE4DC
:103A0000D6018C9391E411969C93119712968C9306
:103A1000D9018E2F90E281111BC0E20FF32FF11D0F
:103A200010828EEF9FEF2996ECE00C94DC219DE252
:103A3000C6CF90E2C4CF2D9381508111FCCFCE0E22
:103A4000D11CE0E0D0CF8EE6D6018C9391E6DBCF9F
:103A50009D938150E0CF482F447082FF3DC084E0A9
:103A6000911101C083E08F1510F4EF2DE81BD601F2
:103A70008E2F20E2552309F1992329F0D6019C933A
:103A8000C60101966C0196012D5F3F4FE2FE1BC0FF
:103A900089E4D6018C938EE411968C93119786E479
:103AA00012968C93D9018E2F90E2882309F4B5CF1A
:103AB0009D938150FACF2D9381508111FCCFCE0E72
:103AC000D11CE0E0D9CF89E6D6018C938EE6119621
:103AD0008C93119786E6E4CF9B0177FF02C030E01C
:103AE00020E0A1E0B0E0911102C0B0E0A0E0F90157
:103AF0003196AE0FBF1F8B2C912CBB2009F461C0F7
:103B00005401EFEFAE1ABE0AAA0DBB1DFA161B0632
:103B100019F014F04F2D4A1B511188C0E3FC59C015
:103B20007601A42FB0E2A1114FC0C40ED11C99237D
:103B300009F45BC040E0D6011196F60190836D0157
:103B4000552309F448C0012F060F9A81582F507150
:103B500084FF03C0913309F4015010160CF047C0E4
:103B6000093008F008E0EEE2FE2E5B01A01AB10871
:103B700085019194819491082F3F320729F4D60151
:103B8000FC92F60131966F016217730794F10217E8
:103B900013077CF5DB01A21BB30BAA24A394B12C61
:103BA000AC0EBD1EAA0DBB1D11968C912150310982
:103BB000D601119628153905F4F0F60180836D01C0
:103BC000DBCFB12CA12CA0CFF701B1937F01A15085
:103BD000AACF9111B0CFD601942F50E302C05D93CC
:103BE00091509111FCCFC40ED11C40E0ACCF01E04C
:103BF000BACF80E3DBCF6217730731F4963388F4D2
:103C0000953311F4552369F0F6018083FD01842F6B
:103C100090E2811108C0A40FB11D1C9290E080E0D9
:103C200002CF81E3F1CF91938150F3CF911183CFF4
:103C30008ACFB0E0A0E0EFE1FEE10C94C0215C018E
:103C40007B016115710519F0DB018D939C93850152
:103C50000F5F1F4FF501D0818D2F90E00E94412012
:103C60006C01892BB9F5DD32B9F50F5F1F4FD50116
:103C70001196DC91C1E05801F1E0AF1AB10843E0C0
:103C800050E060E770E0C5010E944A20892B69F589
:103C9000680182E0C80ED11C45E050E06BE670E0A0
:103CA000C6010E944A20892B21F4680197E0C90EC1
:103CB000D11CE114F10419F0D701CD92DC9260E03F
:103CC00070E080E89FEFC111FFC060E070E080E825
:103CD0009FE7FAC05801BBCFDB3229F485010E5FA4
:103CE0001F4FF501D181C0E0C6CF43E050E068E648
:103CF00070E0C5010E944A20892BE9F0F80110E02C
:103D000000E020E030E0A9015F01B0ED8B2E8D0EC8
:103D100089E08815C8F19C2E689491F88C2F8870E2
:103D2000C2FF16C0811102C00F5F1F4F3196D5012F
:103D3000DC91C92DE9CFE114F10429F00E5F1F4F8A
:103D4000F7011183008360E070E080EC9FE7BCC066
:103D5000882311F001501109A5E0B0E00E94AF21C5
:103D60009B01AC01220F331F441F551F280D311D2D
:103D7000411D511D283999E93907490799E159072A
:103D8000A8F2C6609C2ED2CFAEEF8A1206C0C3FD49
:103D90003CC09C2E689493F8C9CFDF7DD534A9F53B
:103DA00080818D3239F4C061DF011296818162E039
:103DB00070E006C0DF018B32C1F3119661E070E064
:103DC00080535D01A61AB70A8A30F8F4E0E8CE16EF
:103DD000ECE0DE065CF4B601660F771F660F771F16
:103DE000C60ED71ECC0CDD1CC80ED11C5D01FFEF2A
:103DF000AF1ABF0A8C9180538A30A8F1C4FF03C068
:103E0000D194C194D1080C0D1D1DC1FF09C0E1144E
:103E1000F10431F081E0A81AB108D701AD92BC924B
:103E2000CA01B9010E947720C370C33009F49058C9
:103E30004B015C0120E030E0A9010E947220882340
:103E400009F440C0CFE9D0E017FF05C011950195F6
:103E50001109C7E8D0E06E01B8E1CB1AD10880E2C1
:103E6000E82EF12C0FC0D501B1CFFE01259135917F
:103E7000459154910E191F09C501B4010E94D82023
:103E80004B015C01D501C4010E151F0574F7249781
:103E9000F594E794CC16DD06A9F78A2F880F8B2FAF
:103EA000881F8F3F49F020E030E0A901C501B4012F
:103EB0000E947220811106C082E290E09093BD03BF
:103EC0008093BC03C501B401CDB7DEB7ECE00C9420
:103ED000DC21283008F027E03327DA01990F311D63
:103EE00087FD916000966105710539F432602E5F9F
:103EF0003D9330E32A95E1F708959F3F30F08038F5
:103F00007105610509F03C5F3C5F3D93913008F01D
:103F10008068911DDF93CF931F930F93FF92EF92D1
:103F2000192F987F9695E92F96959695E90FFF277B
:103F3000E350FF4F99273327EE24FF24A701E70121
:103F400005900894079428F4360FE71EF81E491FC1
:103F5000511D660F771F881F991F0694A1F70590C2
:103F6000079428F4E70EF81E491F561FC11D770F4E
:103F7000881F991F661F0694A1F70590079428F4DF
:103F8000F80E491F561FC71FD11D880F991F661FA6
:103F9000771F0694A1F70590079420F4490F561F48
:103FA000C71FD81F990F661F771F881F0694A9F790
:103FB00084911095177041F0D695C7955795479500
:103FC000F794E7941A95C1F7E3EAF0E06894159046
:103FD000159135916591959105907FE27395E11862
:103FE000F10A430B560BC90BD009C0F7E10CF11EC7
:103FF000431F561FC91FD01D7EF4703311F48A95DC
:10400000E6CFE894015030F0080F0AF400270217B9
:1040100008F4202F2395022F7A3328F079E37D933B
:104020002A95E9F710C07D932A9589F6069497950D
:104030006795379517951794E118F10A430B560BBE
:10404000C90BD00998F023957E9173957A3308F0C7
:1040500070E37C932013B8F77E9170617D9330F00C
:10406000839571E37D9370E32A95E1F71124EF9036
:10407000FF900F911F91CF91DF91992787FD909528
:10408000089591110C944521803219F08950855082
:10409000C8F70895FB01DC014150504088F08D9134
:1040A00081341CF08B350CF4805E659161341CF01A
:1040B0006B350CF4605E861B611171F3990B0895EA
:1040C000881BFCCFDC01FC01672F71917723E1F79E
:1040D000329704C07C916D9370836291AE17BF07D5
:1040E000C8F308950E94B42008F481E00895E8948C
:1040F00009C097FB3EF490958095709561957F4F30
:104100008F4F9F4F9923A9F0F92F96E9BB279395DD
:10411000F695879577956795B795F111F8CFFAF4ED
:10412000BB0F11F460FF1BC06F5F7F4F8F4F9F4F1E
:1041300016C0882311F096E911C0772321F09EE87C
:10414000872F762F05C0662371F096E8862F70E0E2
:1041500060E02AF09A95660F771F881FDAF7880FBC
:104160009695879597F90895990F0008550FAA0B12
:10417000E0E8FEEF16161706E807F907C0F012167A
:104180001306E407F50798F0621B730B840B950B7D
:1041900039F40A2661F0232B242B252B21F40895D2
:1041A0000A2609F4A140A6958FEF811D811D08956F
:1041B0000E94EB200C945F210E94512138F00E9454
:1041C000582120F0952311F00C9448210C944E2195
:1041D00011240C9493210E94702170F3959FC1F3D8
:1041E000950F50E0551F629FF001729FBB27F00DA5
:1041F000B11D639FAA27F00DB11DAA1F649F6627FA
:10420000B00DA11D661F829F2227B00DA11D621F48
:10421000739FB00DA11D621F839FA00D611D221F02
:10422000749F3327A00D611D231F849F600D211DE6
:10423000822F762F6A2F11249F5750409AF0F1F069
:1042400088234AF0EE0FFF1FBB1F661F771F881FD2
:1042500091505040A9F79E3F510580F00C944821A1
:104260000C9493215F3FE4F3983ED4F386957795C1
:104270006795B795F795E7959F5FC1F7FE2B880F78
:10428000911D9695879597F9089599278827089500
:1042900097F99F6780E870E060E008959FEF80ECF9
:1042A000089500240A94161617061806090608959C
:1042B00000240A9412161306140605060895092E02
:1042C0000394000C11F4882352F0BB0F40F4BF2B71
:1042D00011F460FF04C06F5F7F4F8F4F9F4F0895B1
:1042E00057FD9058440F551F59F05F3F71F04795A7
:1042F000880F97FB991F61F09F3F79F0879508958C
:10430000121613061406551FF2CF4695F1DF08C0AA
:10431000161617061806991FF1CF869571056105C7
:1043200008940895E894BB2766277727CB0197F96F
:104330000895F999FECF92BD81BDF89A992780B56D
:104340000895262FF999FECF1FBA92BD81BD20BDD9
:104350000FB6F894FA9AF99A0FBE019608950E9442
:10436000F121A59F900DB49F900DA49F800D911DEC
:10437000112408952F923F924F925F926F927F92F5
:104380008F929F92AF92BF92CF92DF92EF92FF9265
:104390000F931F93CF93DF93CDB7DEB7CA1BDB0B11
:1043A0000FB6F894DEBF0FBECDBF09942A883988B6
:1043B00048885F846E847D848C849B84AA84B984BD
:1043C000C884DF80EE80FD800C811B81AA81B981C9
:1043D000CE0FD11D0FB6F894DEBF0FBECDBFED01DD
:1043E0000895A29FB001B39FC001A39F700D811DCE
:1043F0001124911DB29F700D811D1124911D0895EE
:104400005058BB27AA270E9418220C945F210E94B3
:10441000512138F00E94582120F039F49F3F19F4BF
:1044200026F40C944E210EF4E095E7FB0C94482101
:10443000E92F0E94702158F3BA17620773078407A7
:10444000950720F079F4A6F50C9492210EF4E095EE
:104450000B2EBA2FA02D0B01B90190010C01CA013E
:10446000A0011124FF27591B99F0593F50F4503EE9
:1044700068F11A16F040A22F232F342F4427585FDB
:10448000F3CF469537952795A795F0405395C9F7F3
:104490007EF41F16BA0B620B730B840BBAF09150AB
:1044A000A1F0FF0FBB1F661F771F881FC2F70EC04A
:1044B000BA0F621F731F841F48F48795779567951D
:1044C000B795F7959E3F08F0B0CF9395880F08F009
:1044D0009927EE0F9795879508950E947422689406
:1044E000B1110C94932108950E94782188F09F5770
:1044F00098F0B92F9927B751B0F0E1F0660F771F08
:10450000881F991F1AF0BA95C9F714C0B13091F0FD
:104510000E949221B1E008950C949221672F782F88
:104520008827B85F39F0B93FCCF3869577956795C2
:10453000B395D9F73EF490958095709561957F4F2E
:104540008F4F9F4F08950E94B42008F48FEF089575
:10455000DB018F939F930E94AF21BF91AF91A29FE8
:10456000800D911DA39F900DB29F900D1124089571
:1045700097FB072E16F4009407D077FD09D00E9410
:10458000D22207FC05D03EF4909581959F4F089567
:10459000709561957F4F0895EE0FFF1F0590F49180
:1045A000E02D0994AA1BBB1B51E107C0AA1FBB1F2A
:1045B000A617B70710F0A61BB70B881F991F5A95AF
:1045C000A9F780959095BC01CD0108950F931F9395
:1045D000CF93DF938230910510F482E090E0E09178
:1045E000C003F091C10330E020E0B0E0A0E03097DC
:1045F00099F42115310509F44AC0281B390B2430E0
:104600003105D8F58A819B816115710589F1FB011E
:1046100093838283FE0111C0408151810281138105
:1046200048175907E0F04817590799F4109761F0B7
:1046300012960C93129713961C933296CF01DF912A
:10464000CF911F910F9108950093C0031093C10360
:10465000F4CF2115310551F04217530738F0A90165
:10466000DB019A01BD01DF01F801C1CFEF01F9CFF4
:104670009093C1038093C003CDCFFE01E20FF31FDF
:10468000819391932250310939832883D7CF209188
:10469000BE033091BF03232B41F420911E013091C2
:1046A0001F013093BF032093BE0320911C01309162
:1046B0001D012115310541F42DB73EB74091200170
:1046C00050912101241B350BE091BE03F091BF03F3
:1046D000E217F307A0F42E1B3F0B2817390778F0D9
:1046E000AC014E5F5F4F2417350748F04E0F5F1F38
:1046F0005093BF034093BE03819391939FCFF0E00B
:10470000E0E09CCFCF93DF930097E9F0FC01329774
:1047100013821282A091C003B091C103ED0130E079
:1047200020E01097A1F420813181820F931F209106
:10473000BE033091BF032817390709F061C0F09319
:10474000BF03E093BE03DF91CF910895EA01CE1736
:10475000DF07E8F54A815B819E0141155105B1F7FC
:10476000E901FB83EA8349915991C40FD51FEC17E6
:10477000FD0761F4808191810296840F951FE90104
:1047800099838883828193819B838A83F0E0E0E030
:1047900012968D919C9113970097B9F52D913C91AC
:1047A0001197CD010296820F931F2091BE03309185
:1047B000BF032817390739F6309751F51092C10316
:1047C0001092C003B093BF03A093BE03BCCFD383AA
:1047D000C28340815181840F951FC817D90761F4A6
:1047E0004E5F5F4F88819981480F591F51834083E5
:1047F0008A819B81938382832115310509F0B0CF93
:10480000F093C103E093C0039ECFFD01DC01C0CF54
:1048100013821282D7CFB0E0A0E0E1E1F4E20C9481
:10482000BC218C01009751F4CB010E94E6228C013F
:10483000C801CDB7DEB7E0E10C94D821FC01E60F4A
:10484000F71F9C0122503109E217F30708F49DC0BD
:10485000D901CD91DC911197C617D70798F0C530D3
:10486000D10530F3CE0104978617970708F3C61BCE
:10487000D70B2297C193D1936D937C93CF010E9464
:104880008223D6CF5B01AC1ABD0A4C018C0E9D1E53
:10489000A091C003B091C103512C412CF12CE12C0B
:1048A000109731F58091BE039091BF03881599054B
:1048B00009F05CC04616570608F058C080911C01EC
:1048C00090911D01009741F48DB79EB74091200152
:1048D00050912101841B950BE817F90708F055C08A
:1048E000F093BF03E093BE03F90171836083A0CF0F
:1048F0008D919C91119712966C90129713967C90C3
:104900001397A815B90559F56C0142E0C40ED11CE6
:10491000CA14DB0420F1AC014A195B09DA011296D2
:10492000159780F06282738251834083D9016D9321
:104930007C93E114F10471F0D7011396FC93EE938C
:10494000129776CF22968C0F9D1FF9019183808359
:10495000F301EFCFF093C103E093C00369CF481692
:10496000590608F42C017D01D3019ACFCB010E9496
:10497000E6227C01009749F0AE01B8010E94C824EC
:10498000C8010E948223870153CF10E000E050CF7E
:10499000FB01DC0102C001900D9241505040D8F75C
:1049A0000895FC018191861721F08823D9F7992772
:1049B00008953197CF010895FB01DC0101900D921C
:1049C0000020E1F70895FB01DC014150504048F020
:1049D00001900D920020C9F701C01D924150504036
:1049E000E0F70895AEE0B0E0E8EFF4E20C94C821FF
:1049F0000D891E898F89988D26E02C831A8309835F
:104A000097FF02C080E090E801979E838D83AE01FE
:104A1000455E5F4F698D7A8DCE0101960E942225F9
:104A20004D815E8157FD0AC02F813885421753079B
:104A30000CF49A01020F131FF80110822E96E4E085
:104A40000C94E421ABE0B0E0E8E2F5E20C94BA218A
:104A50007C013B018A01FC0117821682838181FF60
:104A6000C8C1CE0101965C01F7019381F30193FD6A
:104A7000859193FF81913F01882309F453C18532C9
:104A800039F493FD859193FF81913F01853229F49B
:104A9000B70190E00E941227E7CF912C212C312CF6
:104AA000FFE1F31538F08B3211F190F4803209F107
:104AB000833229F137FC3CC020ED280F2A3050F515
:104AC00036FE20C08AE0989E200D1124922E06C04A
:104AD0008D3291F0803371F7689430F8F30193FDD3
:104AE000859193FF81913F018111DACF21C06894B4
:104AF00031F8689432F8F2CF689433F8EFCF6894C5
:104B000034F8ECCFEAE02E9E200D1124222E68947A
:104B100035F8E4CF8E3229F436FC04C1689436F8B7
:104B2000DDCF8C3619F4689437F8D8CF8836B1F2D7
:104B3000982F9F7D95549330E0F08336A1F1833711
:104B4000C1F1833509F063C02801F2E04F0E511C1A
:104B5000F801C080D180692D70E036FC02C06FEF93
:104B60007FEFC6010E94FC264C01689437F8820151
:104B70000AC00C5F1F4FFFE3F98388248394912CB4
:104B80006501E89437F833FE2DC0522C811491044E
:104B900071F5552009F468CFB70180E290E00E94DA
:104BA00012275A94F6CFF801808189830E5F1F4F38
:104BB000E4CF2801F2E04F0E511CF801C080D180F3
:104BC000692D70E036FC02C06FEF7FEFC6010E94D6
:104BD00007274C018201D5CFB70180E290E00E9407
:104BE00012272A942814190409F0B0F7CECFF60141
:104BF00037FC859137FE81916F01B70190E00E94EB
:104C0000122751105A94F1E08F1A9108BFCF8436C1
:104C100019F0893609F077C0F80137FE6BC0608162
:104C20007181828193810C5F1F4FF32DFF763F2EA0
:104C300097FF09C090958095709561957F4F8F4F34
:104C40009F4F689437F82AE030E0A5010E94422780
:104C5000C82ECA188C2C432C36FE0CC0E89440F8A1
:104C6000C91440F434FE05C032FC03C0F32DFE7EAF
:104C70004F2E892C44FE95C0FE01EC0DF11D808164
:104C8000803309F087C0242D297E422E842D887020
:104C9000582E43FC95C040FE8FC09C2C821418F403
:104CA0002C0C922C981844FE91C0B70180E390E040
:104CB0000E94122742FE09C088E790E041FE02C030
:104CC00088E590E0B7010E941227C91408F48AC051
:104CD000CA94D12C9FEFC91AD90ACA0CDB1CF60161
:104CE00082916F01B70190E00E941227AC14BD04BD
:104CF000B1F74FCF60817181072E000C880B990BA3
:104D00000E5F1F4F92CFD32CE894D4F82AE030E006
:104D1000853739F1232D297FD22E8F3601F148F4C2
:104D20008835A9F0F701868197812B96E2E10C94F2
:104D3000D621803749F08837A9F7D4FE02C068949D
:104D4000D2F820E130E00DC06894D4F8F6CF34FEFC
:104D500003C0822F8660D82E20E132E002C028E016
:104D600030E0F801D7FE0FC06081718182819381AC
:104D70000C5F1F4FA5010E944227C82ECA183D2C68
:104D8000E89437F867CF6081718190E080E00E5F32
:104D90001F4FF0CF42FC02C0839478CF839483945A
:104DA00075CF842D867809F471CFF6CFB70180E2F4
:104DB00090E00E94122783948214C0F3512C73CF89
:104DC000522C5818821408F46ECFF8CF842D8678B0
:104DD00009F47BCF8BE241FE80E247FC8DE2B70114
:104DE00090E071CFB70180E390E00E9412279A947F
:104DF0006CCF8FEF9FEF99CFFC0105906150704011
:104E00000110D8F7809590958E0F9F1F0895FC0193
:104E10006150704001900110D8F7809590958E0FE9
:104E20009F1F08950F931F93CF93DF93182F092F80
:104E3000EB018B8181FD09C01FEF0FEF812F902FB8
:104E4000DF91CF911F910F91089582FF14C02E81A1
:104E50003F818C819D81281739073CF4E881F981D5
:104E6000CF0101969983888310838E819F8101965B
:104E70009F838E83E3CFE885F985812F0995892B60
:104E8000A1F3DACFFA01AA27283051F1203181F1BC
:104E9000E8946F936E7F6E5F7F4F8F4F9F4FAF4F42
:104EA000B1E03ED0B4E03CD0670F781F891F9A1F55
:104EB000A11D680F791F8A1F911DA11D6A0F711D09
:104EC000811D911DA11D20D009F468943F912AE015
:104ED000269F11243019305D3193DEF6CF010895FD
:104EE000462F4770405D4193B3E00FD0C9F7F6CF2E
:104EF000462F4F70405D4A3318F0495D31FD4052F6
:104F0000419302D0A9F7EACFB4E0A695979587958B
:104F100077956795BA95C9F700976105710508956A
:104F20009B01AC010A2E0694579547953795279516
:104F3000BA95C9F7620F731F841F951FA01D0895AE
:104F400011E0CDE0D1E004C0FE010E94CC22219608
:0A4F5000CE30D107C9F7F894FFCF67
:104F5A0047656D696E695F466F63757365725F4217
:104F6A005A5F49525F563800333338000000C20393
:104F7A0080000C0006000300090008000C00040071
:104F8A00060002000300010009005E00BC00770170
:104F9A000000000022028C01B9016F02EA01C80177
:104FAA00DC012563256C752563002563256425636B
:104FBA0000256325732563004F4B00257325632560
:0C4FCA00632573006235353265666400B3
:00000001FF
